:020000040000FA
:10000000073099008316910178308F008312831690
:100010009830810083123130900083160B308500B8
:10002000951611308700831287018501051521304F
:1000300084005E30A00000308000840AA00B1C28E1
:10004000C830A2257F39F0007E30A225031DF017AD
:10005000CA30A225FC39F1005D30A2250339F10434
:10006000CC30A2251C39F2006030A2250339F204FD
:100070006330A225FE007E18F217FE1872177E1D4F
:10008000F2162A30A225F8000030A225F300071E40
:1000900047281126071E47281126071E4728851DB9
:1000A00047280508033A0339031947288A15002809
:1000B00087125B2058280F08F83E031C64288F0025
:1000C000CB0ACC0AC60A5B28051886288518712831
:1000D000051886288518712805188628851871281E
:1000E000A3288F1AB62A8518712803106E190314D5
:1000F000B00D6E113008113A1F390319F9286A3012
:1001000081000B116D1CD2016D1008008F1AB62AE8
:100110000518862803106E1D0314B00D6E153008E7
:10012000113A1F390319F9286D18D2016D140B1DEE
:10013000A0285208F63E0318C82AD201031008006E
:10014000D20A03140800B001D201CA1ECA0ACA1A90
:10015000D02805080339031D6428071AA9280711A8
:100160008711871083160516851608308F008312B5
:1001700029087F390319C5285F080319C528DB0042
:10018000DB0BC028A903071EB828071EC528831645
:1001900078308F00051285128312CC018A15772CD6
:1001A00005080339D8000319D028AA01AC01132689
:1001B0008518AA0A0518AC0A0230AA1BE3280130E8
:1001C000AC1BE328D728AC005719033AA91B013A06
:1001D000A91F023A031DF2280C306C1C0030C70026
:1001E000A91BC7175B204B080319F228ED11D02576
:1001F000F228CA015B206E1330186E175B20301C8A
:10020000942AF3185828EB01A415731D0B29B73055
:10021000A2250319A4112419A411BA016420300CD9
:10022000BA0D6420300CBA0D5B20301C58286420B5
:10023000300CBA0D6420300CBA0D3A08B1003B0600
:100240000F390319EB153C08031931293A060F3908
:100250000319EB153D08031931293A060F39031923
:10026000EB1535223108B2000310B10CAB30A225DA
:10027000310603196B166E1C4529BA1945293A082F
:100280000739FD3E033E031CEB045D22EB08031916
:10029000982935223108B300B20CB30CB20C03100C
:1002A000B30CB20CA830A2253306031D6B12EB0869
:1002B000031998291D22F5213108B3001D22F521CB
:1002C0003108B4001D22F5213108B500B001F1213B
:1002D000F1216420301CC029F121F1217422F52183
:1002E0001D22F5211D22ED21B001E921E921E9219D
:1002F000ED21EB1E7E293608BE00ED166B1F83290B
:100300003708C200ED16EB1F8E29B80DB80D3C3032
:10031000B805450803393804C500ED166B080739E0
:100320000319F9288313623E840039088000F928F4
:100330006E1C9D29EE1FD625EE13EA01731CCC2DF1
:10034000EF103E0D3E39C700C707BE1AC717031985
:10035000AE29FD30C707ED30D8009B25EC133E1BBE
:10036000EC17BC08031DB8294210BE1B4214BE295D
:10037000BD08031DBE294511BE1B4515EC15CC2D2E
:10038000ED213008013A0F39031D5828731DF92853
:100390006B1EF928ED166E1FCF298A150D2D7318C7
:1003A000F9283308C7003408C200B50DB50D3C303C
:1003B000B505450803393504C500EC13321BEC17AD
:1003C000B21BEC17EC156A0AEA00F03E03189829F4
:1003D000F9285B20301C080058285B2030180800E2
:1003E00058286420300CC90C08005B20301C5828A9
:1003F0001030BA073B083A06031D022AA41D022A40
:10040000731887166420300CB10C300CC90C6420B2
:10041000300CB10C300CC90C5B20301C5828642007
:10042000300CB10C300CC90C6420300CB10C300C09
:10043000C90C5B203018080058286420300CB10C1F
:10044000300CC90C6420300CB10C300CC90C5B2092
:10045000301C58286420300CB10C300CC90C6420BE
:10046000300CB10C300CC90C742A5B20301C58289D
:100470001030BA073B083A06031D422AA41D422A3F
:10048000731887166420300CB10D300CC90C642031
:10049000300CB10D300CC90C5B20301C5828642086
:1004A000300CB10D300CC90C6420300CB10D300C87
:1004B000C90C5B203018080058286420300CB10D9E
:1004C000300CC90C6420300CB10D300CC90C5B2011
:1004D000301C58286420300CB10D300CC90C64203D
:1004E000300CB10D300CC90C87123A08103A703933
:1004F000031D7C2A4908B9003A083B060319902AD3
:100500003A083C0603198C2A3A083D06031D0800E8
:100510004908B800EB1708004908B7006B17080036
:100520004908B600EB160800B0185828E921B001B8
:10053000AA224908B200AA224908B300AA224908FF
:10054000B400ED21B001E921E921E921ED218A156D
:100550007811262DED21F121F121ED21F121F1215B
:10056000ED21F121F121ED21F121F129F31CBA2A2C
:10057000781DBC2A8A15112847086E1D803A571924
:10058000803A8039031D582847088039C700CC2D90
:10059000CA01D201D301B001EE1CD401EE10ED1A54
:1005A0005828EF116F136F1277087F39031D6F16EC
:1005B000F81ADD2A740603196F12B2256F19092C77
:1005C00051080319F32AF81AE92A51087406031985
:1005D000F62A510877067F390319F12AF81AA42B55
:1005E000CC2D6F17F62AEF156D156D1D6D11B62503
:1005F000031858285108C900E0390319AE2BC03A36
:1006000003195828F31C5828E03A0319452BC03A1F
:100610000319DB2B603A0319742B203A03198A2B38
:10062000AA25F8181E2B6F1B1A2BEC12491AEC1670
:1006300049121E2B6C13491A6C1749126F1E222B7C
:100640006F1FCC2DEC15EF1049080F39C7000319A7
:10065000412BC70303193F2BC70DC70DC70D7830BA
:10066000C705491A4715F930C707FB30F818FA30A3
:10067000D8009B25471BC70AC71BC703412BEF1494
:10068000C701C713C91AC717662B51083F3A031D84
:100690005828B2255108C900AA25F81C58286F1EF1
:1006A000532B6F1F5828EC15EF104908C7007F39EE
:1006B0000319662BC70347087F390319622B471BB1
:1006C000C70A662BEF14C701C91BC7178030781CF7
:1006D000C7066F1E6E2B8030F71BC7066D1DCC2D15
:1006E000C713A91BC717CC2DAA2540306F1B41305B
:1006F0008400F030800549080F398004F81CCC2DA7
:100700006F1B862BEC12491AEC16CC2D6C13491A70
:100710006C17CC2DAA25491E972B40306F1B4130FA
:1007200084000F308005490EF0398004CC2D433011
:100730006F1B44308400C90DC90D3C30C905000849
:10074000033949048000CC2D51087506031DCC2DBA
:10075000B22551087606031D5828F62A5108511E65
:10076000C22B6F1B5828123AFE39031D5828B401BA
:100770005118B417B22551087F39B404AA25213085
:10078000FF00782DFE39031D5828AA25EF196F198F
:10079000CE2B540AD400FD3E03186F15EE14C7018A
:1007A000A901EC12C001C3016C13C101C401EC1317
:1007B000C201C501CC2D5108B200B2255108B300C9
:1007C000B2255108B400AA256F1B58283208FC39FD
:1007D000EC3A0319FB2B043A031D58286E176F17C8
:1007E00032080339033A0319032C3408F039F03A7C
:1007F000031D58284C2C6E176F1332080339033A27
:100800000319032C4C2C8A1532080F397038B200AA
:10081000402A8F0151083206031DD6015108B2004B
:100820000319192C703AF0390319192C6F11D401DE
:100830005828B6250318582851083306031DD60139
:100840005108B300B62503183A2C51083406031D8D
:10085000D6015108B400AA25D60A5608023A031D4B
:100860005828B21C352C8A15D8296F13321D6F17E2
:100870006E134C2C5308031D5828D60A5608033A09
:10088000031D58283308B4003219492D32080339A2
:100890005504B3006F136E136E1B522C0330FF0010
:1008A000003043250630FF00013043250930FF00AA
:1008B000023043250C30FF00033043250F30FF008A
:1008C000043043256E1B6C2C063033060319602D53
:1008D000073033060319652D1230FF000830432519
:1008E0001530FF000C3043251830FF000D30432534
:1008F0006E1B822C1B30FF00103043251E30FF0082
:10090000113043252130FF00123043252430FF00F1
:10091000143043252730FF00153043252A30FF00CF
:100920001C3043252D30FF00203043253030FF00A0
:10093000213043253330FF00223043253630FF007D
:10094000233043253930FF00243043253C30FF005D
:10095000253043253F30FF00263043254230FF003D
:10096000273043254530FF00283043254830FF001D
:10097000293043254B30FF002A3043254E30FF00FD
:100980002B3043255130FF002C3043255430FF00DD
:100990002D3043255730FF002E3043255A30FF00BD
:1009A0002F3043255D30FF00303043256030FF009D
:1009B000313043256330FF00323043256630FF007D
:1009C000333043256930FF00343043256C30FF005D
:1009D000353043256F30FF00363043257230FF003D
:1009E000373043257530FF00383043257830FF001D
:1009F000393043257B30FF003A3043257E30FF00FD
:100A00003B3043258130FF003C3043258430FF00DC
:100A10003D3043258730FF003E3043258A30FF00BC
:100A2000683043258D30FF00693043259030FF004A
:100A3000703043259330FF00713043259630FF001E
:100A4000723043259930FF00733043259C30FF00FE
:100A5000743043259F30FF0075304325A230FF00DE
:100A600076304325A530FF00773043256E1B422D9D
:100A70001D303306031D422D0030FF00A2256F1FDD
:100A8000B21D6F2D58283306031D08007F08A225CC
:100A90006F2DB2185E2D3218512D2A30FF00A2257D
:100AA0006F2D0130B21D5828330803195828D5007E
:100AB000D5030310D50D0310D50D7C2D3218652DEF
:100AC00008306F1FB21D6F2D582861306F1FB21D87
:100AD0006F2D3408083A031D58288A15752F6F1B8F
:100AE0007E2D6E1FB219782D3406031D58287C2DDB
:100AF0003408FE008A151A2F8A15242FFE003408A8
:100B00000739D900D90AD8010314D80DD90B852D7E
:100B10005808341A942D7E05031D912DB4195828B8
:100B20007C2DB41D58287C2DB419992DFF3AFE0553
:100B30007A2DFE047A2D47087F395807031C0800D8
:100B4000C70A9D2D83169C18A22D9B001C141A0801
:100B500083120800B625031C58285308031D582883
:100B60006D160800B625031C08005828C825D10DAD
:100B7000C825D10DC825D10DC825D10DC825D10D49
:100B8000C825D10DC825D10DC825D10D5108D306D2
:100B90005B206D1CC82D0800D025D201B00158285B
:100BA000ED1AD42D6D1E08008A1578286508033AC1
:100BB000031DDE2D29087F39031D08006708903AC0
:100BC000031D080065089C3E03180800A830A225F4
:100BD000D800AB30A225D8040319080069086804BE
:100BE000031DFB2D6508033A031D08006608703AD3
:100BF000031D0800072EA830A22569067F39031DB2
:100C00000800AB30A22568067F39031D0800EE17E7
:100C1000B2016508B3006608B4006E178A15462D48
:100C2000112600000000000000000000000000008D
:100C300000000000000000000000000000000000B4
:040C400000000800A8
:101000007F240508033903190128AC008E018F01E4
:101010008F18F42A05080339031911282C0603191F
:1010200008280508033903191128AC008E018F0127
:10103000AA01AB010F1A3A2805080339D800031991
:1010400030282C0603191A285808033A03191A28BD
:101050005808AC00AA0A2A08F63E031C1A2867287A
:101060000508033903193028AB0A2B089C3E031CE2
:101070001A286728F31C4028781940288A11BC2AAE
:101080006330AA27003AD70003305719D7065030EB
:1010900006382C1801385718013AA400DE248716A8
:1010A0001730731D731C1530AA27C2001A30731D28
:1010B000731C1830AA27C5002C1CC5102C1845100D
:1010C0004508D718033AC5006C16EF179A2873180D
:1010D000F823F3185E2473192C24A901231785160D
:1010E000DA24ED01ED15E301CA010130AF002F2F25
:1010F0007F224E22EC196C16D8010630AA27F3186D
:10110000D8007319D80029087F39031D5807A0009B
:101110007F30A01BA000CE24241129087F39A41001
:10112000031DA4142410A91B241401305718A4066D
:10113000DE24EF13EF1BA6284510C510EC1FA628D0
:101140000130A91B0230D718033AC504F318C02890
:101150007319EC286C19EC284508D8003C08031DCD
:10116000B52858114218581542294218D815C218E6
:1011700058164219D816C219D817C21B5817422937
:10118000EF1BEC284310C310EC1ECC280130A91B28
:101190000230D718033AC3044410C4106C1FD62879
:1011A0000130A91B0230D718033AC4042430AA27FF
:1011B0006F1E0030D8004105C2005808FF3A4005B4
:1011C000C2042730AA276F1E0030D8004405C5008E
:1011D0005808FF3A4305C504D8016C1E02292D307A
:1011E000AA274518D8043030AA27C518D804A91B47
:1011F000FE283330AA274218D80402295730AA27DC
:101200004218D8043630AA27C218D8043930AA2781
:101210004219D8043C30AA27C219D8043F30AA2763
:10122000421AD8044230AA27C21AD8044530AA2745
:10123000421BD8044830AA27C21BD8044B30AA2727
:101240004519D8044E30AA27C519D8045130AA2709
:10125000451AD8045430AA27C51AD8049030AA27B2
:101260004205031D58109330AA274205031DD810CC
:101270009630AA274205031D58119930AA27420526
:10128000031DD8116630EE1A6930AA27A20058183B
:101290002217D818A216D624230820394038A300D4
:1012A0006C30AA27A304581DCD019C30AA27FF3912
:1012B0000319CD01FF3A4D0703185811581DA31209
:1012C0005819A316DA24D81DCE019F30AA27FF395A
:1012D0000319CE01FF3A4E070318D811D81D071184
:1012E000D8190715581ECF01A230AA27FF390319B4
:1012F000CF01FF3A4F0703185812581E8711581A8A
:101300008715D81ED001A530AA27FF390319D001AF
:10131000FF3A50070318D812D81E8710D81A87141E
:10132000EE12581BEE166E12D81B6E16EF1B11280C
:101330004C08FE3E031C2F2FCC01DE0A31225E0832
:10134000D800D8030319AF29D8030319B429D80347
:101350000319B929D8030319C329DE01CE29243082
:10136000E1002908E000D6292530E1004708E00027
:10137000D6296030E10042080F39E00045186016B8
:10138000C5186016D6296130E100450DE000E00D7A
:10139000F030E005420E0F39E004D6292630E10096
:1013A0000030E000E00DE00D7C30E005E4212F2F5F
:1013B0003408E4003308E0003208E1006314E4215B
:1013C0000022E31D2F2F242F6108E200F221600884
:1013D000E200F221631CEF296408E200F2216310AD
:1013E000851608000830D900E20C0508051685129C
:1013F00003188516DA270512DA27D90BF429080015
:10140000831685168312E311DE01C227DE0ADE1B76
:101410001A2A8316851285168312851A052AC22771
:10142000DE0ADE1B1A2A8316851285168312851E94
:101430000F2AE315831685128312080063117B308F
:10144000E100320E0739E038E400E3106314E421D0
:101450000022E3192F2FE415E3146314E421002282
:101460002F2F5E193B2ADE18382A5E1CCE2CD22C78
:101470005E1CD62CDA2CDE18E62C5E1CDE2CE22C50
:1014800033087C3E031C2F2F3208E1003308E000B4
:101490003408E4006314E42100222F2F73195F2A1B
:1014A000F3185F2A710ED800580C0739DC3EAA27C2
:1014B000D8006E1E642A0310580CD800642A0F301E
:1014C0006E1A8130AA27D8002106031D692AC60199
:1014D0007E2A73196F2AF3186F2A7B08712A093044
:1014E000AA27FF3A4607031C7E2AC60121087F3936
:1014F000FF3A58070318A10A031CA103D22C4B087A
:1015000003190800CB03FA0A7A08F43E031C992A4F
:10151000FA014D08023E031CCD0A4E08023E031C90
:10152000CE0A4F08023E031CCF0A5008023E031C9D
:10153000D00AAF0B7F2A0130AF0047082906803957
:10154000031DC72A6C1EAB2AED1BAB2AED174708FB
:101550007F39031D6D1747082906031DB82A470860
:101560007F39031DED1503196D130319FC017F2A43
:101570004708FF3A29070318C32A6D1FD32AA90A6F
:101580000930E1227F2AA9030C30E1227F2A2908B1
:101590007F39031DC32AA913C71BA9170130AF0048
:1015A0006D13FC017F2A7319D72A73186D178730C2
:1015B000AA2703196D17FF3A7C0703186D17FC0A59
:1015C0007F2AF318E52A731DEE2A6E1A8430AA27A3
:1015D000FF39EF1C03190130AF0008000130EC188F
:1015E000ED1D7B08AF00080005080339033AAC0085
:1015F0008E01BD23C923BD23C923922B8712CD237E
:101600003208113A1F3903192A2B8716C12787126E
:10161000CD233208113A1F3903192A2B8716C12707
:101620008712CD233208113A1F3903192A2B6E1164
:10163000051C6E15050803390319232B0F089C3E62
:10164000031C1A2BA42BCD233208113A1F3903197E
:101650002A2BA42BD801B51958143519D8143518CC
:101660005815B41BD815B41E5816341ED816341D80
:101670005817B41CD8175808B500D801B31F581410
:10168000331FD814331E5815B31DD815B31C581664
:10169000331CD816321F5817B21ED8175808B4007A
:1016A000C830FF003508FE0096277E30FF00FE019F
:1016B000B51B7E14962735087F3903196B2BCA306A
:1016C000FF003408FE0096275D30FF003408033920
:1016D000FE009627872BB51F872BCC30FF003408E0
:1016E000FE00183A1C391C300319FE06962760309C
:1016F000FF0034080339FE0096276330FF00FE0127
:10170000B41B7E14341BFE14B41E7E159627AE3017
:10171000FF007030FE0096270030FF000130FE0011
:101720009627912BBD23BD2370080F3AC900B22321
:1017300070087F390319A02B7108C900B223A32BAD
:101740007208C900B223BD236430DA00C227112811
:101750001830DA00050803392C060319FE2ADA0BC3
:10176000AA2B08000830D800BD23491CBD23491806
:10177000BF27C90CD80BB42B0800A823CA272408FC
:101780000638013AA400DE248716A823A82387126E
:101790000800A823A823A823A82BDA018518E02B8A
:1017A000051CCD2BDA0A0319EE2B0518D22B0310DA
:1017B0006E190314B20DB30DB40DB50D6E11CD2B12
:1017C000DA0A0319EE2B8518E02B03106E1D0314A3
:1017D000B20DB30DB40DB50D6E15CD2B080071080B
:1017E000D800D80C580C0739D23EAA27FB000800B5
:1017F00070087F397F3ABB00BC01BD0172081C39FB
:10180000043A0319082C103A0319082C3B03BC00B6
:10181000EC1472081C39043A0319EC10083A031945
:10182000EC101C3A0319EC106C1172081C39103AB8
:1018300003196C15183A03196C15EF236C10F01B83
:101840006C146330AA27003AD700BA30AA27D80010
:101850006E10D8186E147F2C7E30AA276C10031DD2
:101860006C146330AA27003AD700BA30AA27D800F0
:101870006E10D8186E147310AE30AA27BB00903EBD
:1018800003187F2C7314B130AA27BC00B430AA27E8
:10189000BD00BA30AA27D8005818552C3B08BC0800
:1018A000031DBC07BD08031DBD077F30BB06BC0878
:1018B000031DBC06BD08031DBD067F2C7E30AA2774
:1018C0006C10031D6C140330AA27F4001B30AA27E8
:1018D000F5001E30AA27F6002130AA27F7002A308B
:1018E000AA27F8006330AA27003AD7007F2CCE241D
:1018F000D224D624DA24DE24E224E6242F2FCE2498
:10190000D2241F30D624E030A3056C30AA277319E7
:101910008B2C73181F30A304DA245030A404DE2467
:101920006030AA27033903199A2CF93EAA27A5008B
:10193000E224AE2C7830AA270339A5000310A50DA8
:10194000A50D7530AA270339A5040310A50DA50D13
:10195000A50D7230AA270739A504E2245C30731D57
:10196000731C5A30AA270739A6000310A60DA60D2E
:10197000A60D6030AA2703390319C82C5D30AA27A9
:101980000339A604A60A25080739031DA60ACC2C8C
:101990007B30AA270739A6042617E62C0030A700BB
:1019A0002008EA2C0130A7002108EA2C0230A70009
:1019B0002208EA2C0330A7002308EA2C0430A700F1
:1019C0002408EA2C0530A7002508EA2C0630A700D9
:1019D0002608EA2CA80085148316851005108312AA
:1019E0000730D90005118510051028180514A80C1A
:1019F0008514D90BF32C0330D90085100510271856
:101A00000514A70C00008514D90BFD2C0515C6275D
:101A10008316851405148312080034080319222D37
:101A2000093A0319182D34080A3A0319182D2F2FD3
:101A30008330B418E7303307B3003508B4007F3083
:101A4000B200442AB2013508B400462D0130DA0054
:101A5000320E0739DB000319312D0310DA0DDB0BD1
:101A60002D2D33089C3E03182F2F32080F390319F0
:101A7000462D013A03197C2E083A0319D32E013A58
:101A80000319C82E023A0319CE2E2F2F6E1B502D8C
:101A9000A830FF000130EB26AB30FF000230EB2610
:101AA000AE30FF000330EB26B130FF000430EB26F0
:101AB000B430FF000530EB26B730FF000630EB26D0
:101AC000BA30FF000730EB26BD30FF000830EB26B0
:101AD000C030FF000930EB260930FF000B30EB2649
:101AE0000C30FF000C30EB260F30FF000D30EB26E2
:101AF0000630FF000E30EB268730FF001030EB265B
:101B00008130FF001230EB268430FF001330EB26CB
:101B10007E30FF001530EB262430FF001630EB2618
:101B20002730FF001730EB269030FF001830EB26EF
:101B30009330FF001930EB269630FF001A30EB2669
:101B40009930FF001B30EB261530FF001C30EB26D0
:101B50001830FF001D30EB261F30330603194B2EC3
:101B60002030330603194E2E213033060319512E2F
:101B70002A30FF002A30EB265A30FF003330EB26A4
:101B80006030FF003430EB265D30FF003530EB264F
:101B90001230FF003630EB267230FF003830EB2673
:101BA0007530FF003930EB267830FF003A30EB26F5
:101BB0007B30FF003B30EB262D30FF003D30EB2625
:101BC0003030FF003E30EB263330FF003F30EB2655
:101BD0003630FF004030EB263930FF004130EB2635
:101BE0003C30FF004230EB263F30FF004330EB2615
:101BF0004230FF004430EB264530FF004530EB26F5
:101C00004830FF004630EB264B30FF004730EB26D4
:101C10004E30FF004830EB265130FF004930EB26B4
:101C20005430FF004A30EB265730FF004B30EB2694
:101C30009C30FF004C30EB269F30FF004D30EB26F0
:101C4000A230FF004E30EB26A530FF004F30EB26D0
:101C50006630FF005130EB266930FF005230EB2632
:101C60006C30FF005330EB266F30FF005430EB2612
:101C70008A30FF006230EB268D30FF006330EB26A8
:101C80006E1B4A2E29303306031D4A2E0030FF00FA
:101C9000AA27072F2F2F0430DB00532E0130DB0043
:101CA000532E0230DB006330FF00AA27FE006E1BBC
:101CB0005B2EB21F762E3408FE3E03192F2F5B08D1
:101CC000341C642EFE04672EFF3AFE055B089B273A
:101CD0006E1F6C2E2C242F2F7E08D8000030FF00A2
:101CE0000430FE0096275808FE00B2137E08DB057C
:101CF0000030031D0130072F3308013A03199D2ED0
:101D00003308023A0319A62E3308033A0319A82E02
:101D10003308043A0319AA2E3308053A0319AC2EE6
:101D20003308063A0319AE2E3308073A0319B02ECA
:101D30003308083A0319B22EB42EB21FA42E340869
:101D4000653A0319752F2F2F6130072F1930072F90
:101D50000830072F6530072F0330072F6530072F16
:101D60000030072F0030072F3308D83E03182F2FDD
:101D70003308EC3E031C2F2FE63EFF006E1B2F2F77
:101D8000B21BC42EAA27072F3408FE0096272F2F38
:101D900033089F3E031C2F2F803ED52E3308E73E8D
:101DA00003182F2FD52E3308833EE000E319E62ECB
:101DB000B21F1E2A63191E2A63157F30E100340802
:101DC000E4006314E4210022E3112F2F1027E3180D
:101DD0001027E3112F2F3306031D08006E1BF22E70
:101DE000B21F052F3408FE003127962753276E1F98
:101DF000FB2E2C242F2F7F08D8000030FF0004304A
:101E0000FE0096275808FF00B2137F08AA27B21BCE
:101E10002F2F5A05D80010275808031D15272F2FDC
:101E20000130A4062415A414DE24BE278716BE277D
:101E3000871208003127962753276E1B2E2F00305C
:101E4000FF000230FE0096272415A4140130A406DA
:101E5000DE248716B32787122411DE245E248A111C
:101E600058287F08033A031D392FFE08031D472F0A
:101E70002F2F7F081B3A031D402FC030FE04472F31
:101E80007F082A3A031D472F2730FE05472F7F0A78
:101E9000AA27D8007E06031908007E08FF3A5807D3
:101EA000031808002F2F7F08033A031D5D2F2A30E7
:101EB000FF00AA27DF39FE00962F7F081B3A03197F
:101EC000652F7F081E3A031D6B2F2A30FF00AA27BB
:101ED0002038FE00962F7F08333A031D0800573044
:101EE000FF0096273330FF00080077272F2FFF01D0
:101EF0004130D9009227FF0AFF0AFF0A071E8C2FE4
:101F0000D90B7A2FC8308D27071E8C2FCA308D270A
:101F1000071E8C2FCC308D270800FF00013EAA271A
:101F2000FE00962F7F0A013EAA27FE007F08AA27FF
:101F30007E060319080083169C189B2F7F089B00C0
:101F40007E089A001C1555309D00AA309D009C14F7
:101F50008312080083169C18AA2F9B001C141A08D1
:101F600083120800B727B727B727B727B7276430EA
:101F7000B92FC800DD27C80BBA2F0800C227C22717
:101F8000C227C227C627C627C627C62700000000CB
:101F90000000000000000000000000000000000041
:101FA0000000000000000000000000000000000031
:101FB0000000000000000000000000000000000021
:101FC0000000000000000000000000000000000011
:061FD00000000000080003
:0E1FF2000000000003006500080019006100F7
:02400E00D43F9D
:1042000002000700020003007F00030000000F000F
:1042100000000500FF0005000500FF0005005C0030
:104220007F005C000000010000000100FF000100B1
:1042300003003F000300C000FF00C0000000FF00BB
:1042400000000000FF0000000000FF000000000070
:104250003F0000000600FF0006000100FF00010013
:104260000200FF0002000400FF0004000800FF003D
:1042700008001000FF0010008000FF0080002000F8
:10428000FF0020000000FF0000000000FF00000011
:104290004000FF0040000000FF0000000000FF00A1
:1042A00000000000FF0000000000FF00000004000C
:1042B000FF000400050007000500010003000100E5
:1042C0000200030002000000070000001F001F00A2
:1042D0001F000F001F000F001F001F001F001F0006
:1042E0001F001F000300070003000300030003007A
:1042F00001000300010002000700020000000100AD
:1043000000003F007F003F000100FF0001000000AF
:10431000FA0000000000FF0000000000FF000000A5
:104320000000FF0000000000FF0000000000FF0090
:1043300000000000FF0000000000FA000000000084
:10434000FA0000000000FA0000000000FA0000007F
:1043500001007F0001000A007F000A007000FF00DA
:1043600070000100FF0001000000FF0000000100DC
:10437000010001000000030000000000FF00000039
:064380000000FF00000038
:0C43900001000100BD00BD000600060099
:0C43A400050001000C00030008000200EE
:0443B00010000500F4
:0843B80011004E0038006C00FA
:0843C0002F005C0042007F00A9
:0443CC004C004F0052
:1043D0004B002E002E002E002E002E002E002E0050
:1043E0002E002E002E002E002E002E002E002E005D
:0A43F0002E002E0047003B003900AC
:00000001FF
